:020000040800F2
:10000000F00A0020D9000008B53800084D3000087B
:1000100000000000000000000000000000000000E0
:10002000000000000000000000000000B9380008D7
:100030000000000000000000B7380008BB380008CE
:10004000EB00000800000000EB000008EB000008D7
:10005000EB000008EB000008590D0008630D0008D4
:1000600000000000910C0008A10C0008EB00000843
:10007000EB000008EB000008EB00000800000000A7
:10008000EB0000080000000000000000EB0000088A
:1000900000000000EB000008EB000008EB00000887
:1000A000EB000008EB000008EB00000865430008C7
:1000B000EB0000080000000000000000000000004D
:1000C0000448854600F040FB00480047B146000860
:1000D000C046C046F00A0020044880470448004754
:1000E000FEE7FEE7FEE7FEE7FEE7FEE7AB390008C6
:1000F000C100000830B50B46014600202022012433
:1001000009E00D46D5409D4205D31D469540491B4B
:100110002546954040191546521E002DF1DC30BD94
:1001200070B500242546002801DA01244042002948
:1001300001DA01254942FFF7DDFFAC4200D0404221
:10014000002C00D0494270BD03460B439B0703D0EF
:1001500009E008C9121F08C0042AFAD203E00B788C
:100160000370401C491C521EF9D27047D2B201E004
:100170000270401C491EFBD270470022F6E710B502
:1001800013460A4604461946FFF7F0FF204610BD05
:10019000421C0178401C0029FBD1801A7047F8B539
:1001A00002464A40D40F42004B0052085B089A4274
:1001B00002D20246084611464A0023D0C30D4A0027
:1001C000DDB2120EAD1A202D35DA49020126490A98
:1001D000F6058A19002C00D0524220214F1B1146EF
:1001E000B9402A411018C20D9A4221D0002C17D0D4
:1001F000012D08DCDA05801AD20F8019D207DBB294
:1002000000F009FAF8BDDA05801A012340001B0648
:10021000C01880185A428018CA0F1043490007E0DE
:100220004908C2071143DA05801A8019400880186E
:1002300000F0E9F9F8BD61000122511A001BF7E74F
:100240000122D2075140AAE70122D2075040A6E777
:10025000024670B54A40D30FDB0740002DD04A005C
:100260002AD0010E140E000212020919400A520A85
:100270008418E50104465443000A120A2E04504330
:10028000A4194219200CC543AA18120C0125AD036C
:10029000521C521912047F39240400D0521C1043FE
:1002A00001D44000491EC2B20C06C0092018401CEF
:1002B0004008802A02D003E0002070BD40084000C2
:1002C000002900DA0020184370BD420005D042002A
:1002D000120E52428A4201DB00207047C9050818FD
:1002E00070470000F0B507460846584087B0C00F79
:1002F000049048000E46590040084908BC1A88413D
:1003000005D2384631461E4617460B46024658006F
:10031000400810434DD0300D039040055900400D6A
:10032000490D0590401A0290402873DA1803012104
:10033000000B09050843019004980092002806D09C
:100340001146019A49420020904100910190029883
:1003500040210A1A0199009800F032F905460C462E
:100360006B4607CB00F03CF9C0197141039A0E0DA2
:100370000023D71756401A467A40164344D0049AB1
:10038000002A2DD0029A012A039A15DC1205C01A00
:10039000914101263605001C7141D20F059ED207FE
:1003A0000093019202962A46234600F07AF907B09C
:1003B000F0BD38463146FAE71605234A0F46B21813
:1003C000C01AB74101210905001C4F4100187F41A7
:1003D000114618187941E20F10436D19644113E07A
:1003E000E2076D0815436408C2071443039A012607
:1003F0001205C01A91413605001C7141CE07400814
:1004000030434908C01851412A46234600F03CF9C0
:10041000CDE7FFE7049801224000C117121A00231C
:100420008B4104983146C417381AA141EEE730B425
:100430000124E407634030BC54E730B40124E407EE
:10044000614030BC4EE700000000E0FFF0B51FB493
:1004500088B00B990998002448400999C00F4900B9
:1004600049080991C0070B990090490049080B9170
:1004700009990898A64608431CD00B990A98084386
:1004800018D0099801244000420D4800410D0998F8
:1004900024050003000B204309900B980003000B78
:1004A00020430B9050181C4940180022019014461C
:1004B000104605E0002001460DB0F0BD032801DA2A
:1004C000034600E003239C46C11A0AAE0AE05F001F
:1004D00008ADED5B4F00F75B7D430027AA187C4118
:1004E000491C5B1E6145F2DD410004AB5A522104F8
:1004F000120C0A43240C401C0828DFDB01980290F0
:100500000099704601910090059B049A07990698FE
:1005100000F0C7F8D0E700000DFCFFFF10B5002287
:100520009623114600F077F810BD00000EB5C217F3
:10053000C10F5040CA0740180021054B0293019299
:1005400000910A460B4600F0ACF803B000BD000075
:10055000330400000EB505490291002100910A46BE
:100560000B46019100F09DF803B000BD330400007C
:10057000410040020122400AD205090E80187F295D
:1005800001DA00207047962903DC9622511AC840F0
:10059000704796398840704710B5002904DB012464
:1005A000E40740428C412146002B04DB1C4601231A
:1005B000DB075242A341994200D1904210BD000096
:1005C00010B5202A04DB0146203A9140002010BDDE
:1005D000914020239C1A0346E3401943904010BDEC
:1005E00010B5202A06DBCB170846203A1041C11768
:1005F0000B4306E00B461341D0402024A21A914041
:100600000843194610BD002904DA401C490001D1F5
:1006100040084000704770B40024050C05D1102438
:10062000000402D1002921D01124050E01D10002BD
:100630000834050F01D10001241D850F01D1800070
:10064000A41C002801DB4000641C002908D02025E0
:100650002E1B0D46F540A14000D00121294308433F
:1006600001061B1B000ADB1D02D5002070BC704771
:10067000DB05181880180029F8DA401C4900F5D16C
:1006800070BC40084000704710B5002B08DA002409
:10069000401C614192185B411A4301D1400840005F
:1006A00010BDF0B51FB482B005460C0003D008465B
:1006B00003F0ECFE02E003F0E9FE20300246009079
:1006C00021462846FFF77CFF049B059A04460F4607
:1006D00018431143084314D0184610431BD0009808
:1006E00040210A1A1846059900F040F805460E46C2
:1006F000009A05990498FFF763FF084305D001208D
:1007000004E02046394607B0F0BD0020C11705437C
:100710000E432C43374300990E986305401A790520
:10072000E40A00220C43FD0A0A3002D500200146EB
:10073000E9E70105101969410C9C0D9D00196941FB
:10074000FFF7A2FFDFE70000064C0125064E05E09B
:10075000E36807CC2B430C3C98471034B442F7D3E2
:10076000FFF7B2FC184C0008384C000810B5202ADE
:1007700004DB0846203AD040002110BD0B46D34090
:10078000D0402024A21A91400843194610BD000011
:1007900070B50446006802F077FD002824D0206878
:1007A00081688907C90F04D18168104A114010314E
:1007B000816001F07DFA054612E001F079FA401BF4
:1007C00002280DD920688068400709D5A06D102146
:1007D0000843A065E06D01210843E065084670BD4F
:1007E000206880684007E8D4002070BDE8FFFF7FE4
:1007F00010B5846AA16D502211420DD1A06D012166
:1008000049020843A065206802F042FD00281AD082
:10081000A07E002807D016E0A16DC90623D520468A
:1008200000F02CFC10BD2068016809070BD502F010
:100830002BFD012200280AD0A06D20210843A065CD
:10084000E06D1043E065204600F016FC10BD206806
:1008500041680C2399434160A06DFF210131884319
:100860001043A065EFE7216D496B884710BD10B5B7
:10087000806A816D402211438165C16D042211435C
:10088000C16500F0FBFB10BD10B5806A00F0F5FB00
:1008900010BD0000F8B50446006881688907CD0FD7
:1008A00002F0EEFC00282AD0002D28D120688168B3
:1008B0000522114010260127012914D18168114A0F
:1008C0001140891C816021680320086001F0F0F963
:1008D000054610E001F0ECF9401B02280BD9206816
:1008E0008068C00707D0A06D3043A065E06D384335
:1008F000E0650120F8BD20688068C007EAD10020CB
:10090000F8BD0000E8FFFF7FF8B504460020009026
:10091000206802F0B5FC002845D120688168234A90
:1009200010271140002930D18168D6433140491C3D
:1009300081601F48006807218905084000020AD528
:100940001D481C490068FFF7D5FB401C00E0401E15
:1009500000900028FBD1607E012824D001F0A8F986
:1009600005461BE002F08CFC002804D12068816859
:100970003140491C816001F09BF9401B02280DD9D0
:1009800020680068C043C00708D0A06D3843A06548
:10099000E06D01210843E0650846F8BD2068016864
:1009A000C943C907DED10020F8BD00001700008050
:1009B00008270140400D03005C00002010B52D4CBD
:1009C000012023881A464100615A994201D90B46F9
:1009D00002E0914200D20A46401CC0B2FA28F2D38B
:1009E000981A254C002802DDE18C4018E084E0795B
:1009F000411CE17104283BD326200521205EFFF72E
:100A00008FFB1E4948431E49FFF78AFB1A21615E8E
:100A100000B248430A21FFF783FBA18B4118012054
:100A200020564843E0842082E078012803D0E07813
:100A3000002803D004E0208A608201E0208AA0829E
:100A40000020E084E0711220205E0E494018490029
:100A5000884201D996200AE01220205E7D21FF30D5
:100A6000C900F530884201D9642000E02820E082E6
:100A700010BD0000E001002000000020E40C000098
:100A8000FF0F0000DC050000F8B504464088002593
:100A90000A3080B2022160800A2802D96279002AD5
:100AA0000AD0962802D96279012A13D0E1888842B7
:100AB00001D965716580F8BD012060713320207215
:100AC00065720091234621780833AC22204600F05D
:100AD00095F8F8BD61710720009023461C332178FA
:100AE0001E460022204600F04CF82079002802D053
:100AF00025636563F8BD0621304600F0AEF8254653
:100B00002035A9788842F5D1207F982108401828FF
:100B1000F0D1607FA17F00020818E67F0002301844
:100B20000009FFF7FBFC0E49FFF792FB1327FF4379
:100B30003946FFF7CAFB206330072978000D0818F3
:100B4000697800020818FFF7E9FC0649FFF780FB07
:100B50003946FFF7BAFB0449FFF772FB6063F8BD43
:100B60000000C842000048430000484202700022D2
:100B70004271FF22F532914201D9C1807047C28093
:100B80007047FFB581B0039800244F000A9D1E46B0
:100B9000002813D002F007FBF8B202F0D4FA02F0FA
:100BA00043FB012800D10124039802F0CCFA02F0A3
:100BB0003BFB012800D1641C02F015FB02F0F3FAA4
:100BC0007F1CF8B202F0BFFA02F02EFB012808D118
:100BD000641C06E06D1EE8B202F085FA3070EDB2DA
:100BE000761C002D03D0002C01D1142DF2D302F07D
:100BF000FAFA01980471204605B0F0BDFFB581B046
:100C00001E460F4600250A9C02F0CDFA7806000E1B
:100C100002F099FA02F008FB012800D1012503989F
:100C200002F091FA02F000FB012809D16D1C07E0E7
:100C3000307802F088FA02F0F7FA641EE4B2761C0B
:100C4000002D03D1002C01D0142CF1D302F0CBFAEB
:100C5000019928460D7105B0F0BD70B50446FF201E
:100C60000023312510E0227850400022060602D5EC
:100C70004000684000E04000521CD2B2C0B2082AD6
:100C8000F4D35B1CDBB2641C8B42ECD370BD000060
:100C900010B5024800F0B6FC10BD0000D0040020E2
:100CA00010B5034800F0AEFC024800F0ABFC10BDEC
:100CB0001C0600207806002010B50446006C094987
:100CC0008008800040186064207814210838FFF7FD
:100CD00011FA04498031A164C106C90E012088407F
:100CE000E06410BD000802400179084B8906890EB6
:100CF0008A00D2180265054A4432491E42658A07B5
:100D0000920F01219140816570470000FC0802406C
:100D1000F0B5846CC56C6560046D002C02D0446D28
:100D2000856D65600B4F7C68056C1C26354001267F
:100D3000AE4034437C60046863608368102B0368B2
:100D400003D099600068C260F0BD9A600068C1601D
:100D5000F0BD00000000024010B5082000F052FE77
:100D600010BD10B5802000F04DFE10BD72B6FEE73C
:100D700003494A6901231B04184302434A6170472F
:100D800000200240044A5069044BC9001840014346
:100D900003480143516170470020024007E0FFFF14
:100DA0000200010030B505494C6901252C434C6116
:100DB0000260BFF36F8F436030BD0000002002402F
:100DC00030B50B4C002263690125AD042B436361F0
:100DD000EFF3108372B620C9521C20C0D2B2402A51
:100DE000F9D32069C003FCD483F3108830BD000020
:100DF00000200240F8B5074600F05AFFC51901244B
:100E00002404114E03E000F053FFA84214D23069CD
:100E10002042F8D130690D4908400D49316103D0B5
:100E20000C4948600120F8BD00F042FFC41905E0FC
:100E300000F03EFFA04201D30320F8BD306940031B
:100E4000F6D40020F8BD000000200240FA83000024
:100E5000FB830000D4060020FEB504460020264691
:100E60000190403600900127307DFF070D46012894
:100E700010D001203075206802F006FA00280BD04F
:100E8000A06D20210843A06501200190002030754D
:100E90000198FEBD0220FEBD686802287ED021694F
:100EA000B94202D06D4A914207D120682968826A0E
:100EB0004903490B0A4382626DE0C3060F22DB0E31
:100EC0001046216E984081432868470302D0C70727
:100ED0004BD102E04000C00E48E0870701D5012059
:100EE00044E0470701D5022040E0070701D5032071
:100EF0003CE0C70601D5042038E0870601D505206F
:100F000034E0470601D5062030E0070601D507206A
:100F10002CE0C70501D5082028E0870501D5092068
:100F200024E0470501D50A2020E0070501D50B2064
:100F30001CE0C70401D50C2018E0870401D50D2062
:100F400014E0470401D50E2010E0070401D50F205E
:100F50000CE0C70301D5102008E0870301D511205C
:100F600004E0400301D5122000E000209840014336
:100F700021666968E3698808401C98420BD820689C
:100F80002F68836AC906C90E8A409343BA00120FBC
:100F90008A40134383622068AA6800E037E029682A
:100FA000436909028B431140490149090B434361DD
:100FB0002A68002A00DB69E72948016807239B05A6
:100FC0001940284B9A4213D10B0211D4D20211437B
:100FD00002F066F9254824490068FFF78BF80C21D8
:100FE000401C484300E0401E00900028FBD14DE724
:100FF0001F4B9A4203D1CB0101D4920205E01D4B55
:101000009A42D8D14A02D6D45A02114323E0206929
:10101000B84202D01149884206D120682968826A04
:101020004903490B8A4382622A68002AC3DA0C48C2
:10103000016807239B0519400A4B9A4201D1D2024D
:1010400008E00B4B9A4201D1920203E0094B9A420D
:10105000B1D15202914302F023F917E70400008056
:1010600008270140001000B0400D03005C00002084
:10107000004000B8002000B470477047704700007F
:10108000FEB50026044602963746019600960028D3
:1010900005D02546A06D2035002802D007E00120AC
:1010A000FEBD204600F0FCF8E76554200755206897
:1010B0008168C900C90F12D18168724A11400122AA
:1010C00012071143816071486F490068FFF712F8F9
:1010D0004000801C00E0401E00900028FBD12068EA
:1010E0008168C900C90F08D1A16D10221143A16503
:1010F000E16D01221143E165164602F0C5F8A16DCC
:10110000C90601D4002804D0A06D10210843A065B1
:10111000B4E0A06DFF210131884302210843A0659E
:10112000206802F0ADF800286DD1217EA068890307
:101130000843617EA27EC903530319430843216B10
:10114000002901D0012109030843E168084321690E
:10115000002902DA4900490801E001214905084354
:10116000297B49000843029908432978012909D1BC
:10117000002A22D0A16D20221143A165E16D012238
:101180001143E165616A002906D0FF23C13319408C
:10119000A26A0143104608432168CA683C4B1A40C2
:1011A0000243CA606168019A890F8907E06C0A43AB
:1011B00010432A7F012A04D00CE0012109040843CE
:1011C000E0E7636C226C491C1A43A36C0B43114685
:1011D0001943084321680A692E4B1A4002430A61E9
:1011E00003216068890788420DD0590788420AD0D8
:1011F0004900884207D0284A91680F239B049943ED
:101200001840014391600021626B206802F04FF8A2
:101210002249A26B206802F04AF80F212069C943D5
:1012200000281CD00122520590420AD12068826A0F
:10123000227F9200121FD206D20E9140226E1143DD
:10124000816220684069616B4007400F88420BD182
:10125000E765A06D80088000401CA0650FE0206855
:10126000826A0A438262ECE7A06D02218843102162
:101270000843A065E06D01210843E0650126304682
:10128000FEBD0000E8FFFF7F400D03005C00002072
:101290000102FEFF02FCFF1F0027014004FFFF07C1
:1012A00070B58CB0054614216846FEF766FF18211C
:1012B00005A8FEF762FF24492868884242D1012030
:1012C000800305904004099005A800F09BFD0028CC
:1012D00001D0FFF74BFD1D480268012109050A43B3
:1012E0000260006808400B9018484038416B0122AA
:1012F00011434163406B002610400B900220009088
:1013000003200190052069460296000700F01CFCAE
:10131000104C0F482060A6600520E66060608020C9
:101320002061400060618000A0612020E061C00178
:101330002062204600F0C2F9002801D0FFF716FD18
:101340002C65A5620CB070BD002401404010024025
:1013500008000240D0040020F7B50446006801F000
:1013600093FF002845D125464035287D012840D0EF
:1013700001272F752068C1681F4EC9070CD101F0E5
:101380007FFF002804D0206881683140891C81607B
:101390002068C1683943C1602046FFF7B5FA0028CC
:1013A00026D1A06D15490840FF2101310843A065F1
:1013B0000020E065226D1249D162226D114911634E
:1013C000226D1149516322681C2111602875206823
:1013D00041681022114341602168206D4031029B19
:1013E000019A00F0BDF921688A683240121D8A60B6
:1013F000FEBD0220FEBD0000E8FFFF7FFEF1FFFF03
:10140000F1070008890800086F080008F8B50646CB
:1014100004464036307D012807D001273775204625
:10142000FFF7B6F9050002D028E00220F8BD206DD4
:101430002521095C022907D100F024F8050003D01A
:10144000A06D40210843A0652068416810229143A7
:101450004160002D204602D0FFF71CFA09E0FFF79B
:1014600019FA050005D1A06DFF21013188433843E9
:10147000A0652068C16849084900C1600020307536
:101480002846F8BDF0B5002808D0014620314A7939
:10149000022A05D00422C263002008710120F0BD99
:1014A000026813680E24A3431360426C1468FF2380
:1014B00001339C431460026814686408640014607B
:1014C0000C4E7268056C1C24254001242746AF4051
:1014D0003A437260826CC56C5560026D002A05D07B
:1014E00015689D431560826D406D42604C7100200F
:1014F0000871F0BD00000240F8B50024014620311B
:101500004A79022A03D00421C16301242DE0026834
:1015100013680E25AB431360026813685B085B0019
:101520001360426C1368FF250135AB431360104E06
:101530007268056C1C231D4001231F46AF403A43CF
:101540007260826CC56C5560026D002A06D0166808
:101550001D02AE431660426D856D55604B710022D1
:101560000A71816B002900D088472046F8BD000031
:101570000000024070B5040038D0206801684908B6
:10158000490001601A48266814213018FEF7B2FDA0
:101590008000002520643560164B5868216C1C22A1
:1015A000114001228A40104358602046FFF784FB17
:1015B000606C0560A06CE16C41606068401E0328AF
:1015C00007D82046FFF790FB206D0560606DA16D88
:1015D000416025656565A565E56225636563A5636D
:1015E000E563203465712571002070BD012070BD58
:1015F000F8FFFDBF00000240C06B7047203040790B
:1016000070470000F0B42C4D2B6801680A68046C28
:101610001C273C400426A6401E4211D056070FD579
:101620000A68920603D40B68042293430B606A682D
:10163000036C04213B4099400A436A60016B1CE043
:101640000227A74006461F402036002F19D09707D3
:1016500017D50A68920605D40A680A239A430A60D5
:10166000012171716B68026C1C210A4002219140BA
:101670000B436B6000213171C16A00291AD0F0BCA4
:1016800008470827A7401F4214D0120712D50A683E
:101690000E239A430A606A68036C1C210B400121E7
:1016A0000C469C4022436A60C16371710021317114
:1016B000416BE2E7F0BC70470000024070B50400E7
:1016C0003FD02548256814212818FEF713FD800017
:1016D0002064022026462036707128681F49084081
:1016E0002860A168E06862690143206910430143F2
:1016F000A0690143E0690143206A01432068026850
:10170000114301602046FFF7D7FA0121A068890341
:101710000025884200D165602079616C8006800ECA
:101720000860A06CE16C41606068401E03280AD824
:101730002046FFF7D9FA206D0560606DA16D41600C
:1017400004E0012070BD25656565A565E5630120A0
:1017500070713571002070BDF8FFFDBF0F80FFFF75
:10176000F8B504468C4620300179002501290BD0BC
:101770000126067147790021012F07D08022E263FC
:10178000017101252846F8BD0220F8BD02274771E6
:10179000E16320680168490849000160614620460C
:1017A000FFF7B6FA206B00282068016801D00E22EE
:1017B00005E0042291430160206801680A22114378
:1017C0000160606C0168084AC90302D501681143D1
:1017D0000160206D002802D001681143016020687B
:1017E000016831430160CDE700010000F8B51F4FEB
:1017F000044638780E4601280AD0012038700020AF
:1018000078607D20C000FFF7F5FA002802D029E0BB
:101810000220F8BD042161602268042A03D0491F18
:101820003160A56814E00846FFF7A2FA7D20C000E9
:10183000FFF7E0FA16E029466068FFF7A3FA7D207B
:10184000C000FFF7D7FA002801D0356005E06D1C15
:10185000E268A1688918A942EDD805494A690223BE
:101860009A434A6100213970F8BD0000D406002077
:1018700000200240054901204A69C3071A434A6112
:101880004969002900DA002070470000002002406A
:10189000F0B51FB4144E05463078144601280AD01E
:1018A0000120307000277D20C0007760FFF7A2FA8A
:1018B000002803D010E0022005B0F0BD012D0DD0AE
:1018C00021460198FFF77CFA7D20C000FFF792FACD
:1018D00006494A69AA434A613770EDE72246039BED
:1018E0000198FFF75FFAEFE7D406002000200240DE
:1018F000064900204A69002A07DA054A8A60054A33
:101900008A604969002900DA0120704700200240FE
:1019100023016745AB89EFCDF0B5002255E00123E7
:1019200093409E460B404FD095082A4CAD002C1991
:10193000256E9607F70E0F26BE403540AC460525AE
:101940002D07A84201D100250FE0234DA84201D167
:1019500001250AE0214DA84201D1022505E0204DD4
:10196000A84201D1032500E00525BD40654511D100
:10197000184D80352F689F432F606F689F436F60BD
:10198000144D6F689F436F602F689F432F60236ED5
:10199000B3432366046855000323AB401C43046033
:1019A000D408A4002418266A5507EF0E0F25BD4061
:1019B000AE43266284689C43846044687546AC43A9
:1019C0004460C4689C43C460521C0B46D340A6D1FB
:1019D000F0BD000000180240000400500008005054
:1019E000000C005010B5082808D105200821000778
:1019F00000F04AF9002801D10149C87010BD00006B
:101A00000000002070B5084D0446E868204203D06D
:101A1000EC60204600F00AF82869204203D02C61CF
:101A20002046FFF7DFFF70BD00180240F8B505271C
:101A300005463F074021384600F026F93F4E8021F9
:101A4000B072384600F020F90024F072802D02D0E8
:101A5000082D2FD06EE001286CD100F029F907463F
:101A6000F06A381A08280DD27D21C900042002F03E
:101A7000A1FD3079012805D1FF21F531022002F0C6
:101A800099FD3471F762B07A012802D1707A401C56
:101A90007072307A401CC0B230720A284AD3707A11
:101AA000032801D3012001E00020C043707034728C
:101AB00074723FE02249032002F07CFD0821384681
:101AC00000F0E2F8012835D10122F2701220305ED8
:101AD0001421715E401A1623F35E032198420BDD38
:101AE000307B401CC0B230737473032800D3B470D1
:101AF000FA280CD931730AE0707B401CC0B27073B5
:101B00003473032800D3B270FA2800D971732422E9
:101B1000B25E0A2A0EDB1221715E002900DA494208
:101B2000914207DA1420305E002800DA40429042E9
:101B300000DAB4700348C560F8BD00000000002062
:101B40008813000000180240F0B500228EE0012545
:101B500095402B407ED00C79A407A40F012C01D016
:101B6000022C10D1866854000327A740BE43CF68DB
:101B7000A740374387604468AC430D79ED06ED0F0D
:101B80009540254345600C79E443A40708D0C56817
:101B900054000326A640B5438E68A6402E43C66077
:101BA0000C79A407A40F022C0CD1D408A400271888
:101BB0003D6A5407E40E0F26A640B5430E69A640C1
:101BC0002E433E62056854000326A640B5430E79B5
:101BD000B607B60FA6402E4306604C68A403A40FB8
:101BE00043D09508244CAD002F193D6E9407E40EA8
:101BF0000F26A640B54305263607B04201D1002680
:101C00000FE01E4EB04201D101260AE01C4EB04248
:101C100001D1022605E01B4EB04201D1032600E0AF
:101C20000526A6402E43144D3E662C684E689C4304
:101C3000F60200D51C432C606C684E689C43B602CB
:101C400000D51C436C600C4D80356C684E689C431D
:101C5000B60300E009E000D51C436C602C684E68B8
:101C60009C43F60300D51C432C60521C0B681C4699
:101C7000D44000D06BE7F0BD0018024000040050D3
:101C800000080050000C00500069084000D00120FE
:101C90007047426913460B401B0491430B43836119
:101CA0007047002A01D0816170478162704700004F
:101CB0000148806870470000500000200068024919
:101CC0000160002070470000AAAA00000248816855
:101CD00002788918816070475000002010B50848CC
:101CE00000240168821511430160032000F00AF806
:101CF000002801D0012401E000F028F8204610BDA2
:101D00000020024070B50F4E0024317805460029AE
:101D100015D07D20C000FEF7EDF901460A480068A5
:101D2000FEF7E8F900F00CFC002808D1042D06D2DB
:101D300000222946401E00F03BF8756000E00124B7
:101D4000204670BD500000205C00002008B5094806
:101D500001680122114301600068104000900548AD
:101D60004038C26B01040A43C263C06B0840009054
:101D700008BD000040100240002809DBC106C90E62
:101D80000120884003490860BFF34F8FBFF36F8F76
:101D90007047000080E100E0002805DBC106C90EA5
:101DA00001208840014908607047000000E100E020
:101DB00010B502F083FB10BD10B50F4C2168032253
:101DC0005202914301432160C11FFF39FA390ED1FC
:101DD0000A480621006848430949FEF78BF9401C70
:101DE00002E0002805D0401E61694905F9D40020B1
:101DF00010BD032010BD0000007000405C000020FA
:101E000040420F00FEB5044600250068524E2F46A2
:101E1000800359D5002001904F484038C06BC00066
:101E20000AD44D484038C26B01040A43C263C06BF8
:101E30000840009001200190484801688215114334
:101E40000160FFF735FF009007E0FFF731FF0099D1
:101E5000401A022801D903252CE040480068C0053B
:101E6000F3D5002D26D1F0690321090208400FD0D7
:101E7000616981420CD0F06903210902F26988434B
:101E8000012109040A43F261F2698A43F261F061B7
:101E9000C00759D0FFF70CFF009006E0FFF708FFDE
:101EA0000099411A2E488142D5D8F0698007F5D5AE
:101EB000002D49D02F460198002805D026484038EB
:101EC000C26B01048A43C2632078C00705D07069E1
:101ED000616880088000084370612078800606D51C
:101EE0007069032109038843A16808437061208851
:101EF000400411D570692169800080080843706131
:101F0000012120698907884206D113484038C168F9
:101F1000012212041143C1602088000512D57069A6
:101F2000032189038843E168084370610121E06867
:101F30008903884206D108484038C168012212044A
:101F40001143C1603846FEBDF06903210902884390
:101F500061690843F061AEE7401002400070004044
:101F600088130000F8B50D46040044D04D480068C1
:101F70004007400FA84214D24A4F3868C008C0003A
:101F800028433860FFF794FE064605E0FFF790FE11
:101F9000811B4548814260D838684007400FA842FD
:101FA000F4D12068414E81070DD5400704D5B068B3
:101FB000072109030843B060B0680F210902884374
:101FC000A1680843B0602078C00731D0606801285C
:101FD0000AD002280BD000280FD034494031032802
:101FE0000ED0C969890704E03168890301E03168CE
:101FF0008901002906DB0120F8BD31684905F8E7B1
:10200000096AEFE7B168C908C9000143B160FFF789
:102010004FFE074605E0FFF74BFEC11B22488142F9
:102020001BD8B068382108406168C9008842F2D1E5
:102030001C4801684907490FA94216D90168C90817
:10204000C90029430160FFF733FE074607E0FFF7A9
:102050002FFEC11B1448814201D90320F8BD11484D
:1020600000684007400FA842F1D12078400706D50C
:10207000B168072000038143E0680143B16000F0CC
:1020800031F8B1683C2289091140094A515CC906FE
:10209000C90EC8400749086007480068FFF732FECC
:1020A000F8BD00000020024088130000001002402C
:1020B000B84B00085C000020540000200648074987
:1020C00000688968064A4904490F8900515CC906BD
:1020D000C90EC840704700005C000020001002409C
:1020E000F84B000810B5204CA068204A8006400F2D
:1020F00016D0A0688006410F501001290FD0A168AA
:102100008906490F022912D0A0688006400F0428D2
:1021100023D0A0688006400F032821D0002010BDE6
:10212000206801218004400F8140104612E0E168E0
:102130008B07E1689B0F4906490F491C032B00D010
:102140001046FDF7D7FFE1684904490E4843E168AE
:10215000490F491CFDF7CEFF10BD0120C00310BD83
:102160007D20000210BD0000001002400024F40099
:10217000F8B504007ED020783827C007E74E002845
:1021800045D0B068F16838408907890F102802D01F
:1021900008280AD001E0032907D00121606809045A
:1021A000884209D13068084314E0306880032ED596
:1021B00060680028DED02AE0052301221B04920477
:1021C0009842306802D110433060EBE788433060BA
:1021D000306890433060606800280CD0FFF768FDDD
:1021E000054604E0FFF764FD401B642873D830689F
:1021F0008003F7D50BE0FFF75BFD054604E0FFF732
:1022000057FD401B6428F1D830688003F7D420784C
:10221000800769D5B068F16838408A070721920FB6
:10222000C902102802D0002813D001E0022A10D0E1
:10223000E068002846D03068884321690843306050
:102240003168FF20013001433160FFF731FD054661
:102250002CE03268520502D5E268002A8AD0726802
:102260007F231B029A4363691B021A437260002892
:1022700010D100E08DE03068884321690843306068
:10228000306801218004400F8140A548FDF732FFEE
:10229000A4490860A4480068FFF734FD002878D1FD
:1022A00022E0FFF705FD401B02289FD8306840055B
:1022B000F7D570687F2109028843616909020843E4
:1022C000706011E03168FF20013081433160FFF719
:1022D000EFFC054605E096E0FFF7EAFC401B02280C
:1022E00084D830684005F7D42078904D00072ED56B
:1022F000B0688006400F03280AD0A0690028286A29
:1023000016D0012108432862FFF7D2FC07460BE0F4
:10231000286A80071BD5A06900289FD017E0FFF727
:10232000C7FCC01B02286ED8286A8007F7D50EE0CC
:10233000400840002862FFF7BBFC074604E0FFF7B7
:10234000B7FCC01B02285ED8286A8007F7D4207823
:1023500040076AD500200090B0688006400F04282E
:1023600018D0F06BC00008D4F16B012000070143C6
:10237000F163F16B0140012000906D480168C905CF
:1023800018D4026881150A430260FFF791FC0746E2
:102390000CE083E0E869800747D5A06800287DD07D
:1023A00043E0FFF785FCC01B02282CD8604800687A
:1023B000C005F6D5A068012810D004210528E869D9
:1023C00010D040084000E861E8698843E861A068EF
:1023D000002814D0FFF76CFC07460CE0E8690121E7
:1023E0000843F3E70843E861F8E7FFF761FCC11B26
:1023F0005048814265D8E8698007F6D50DE0FFF7BF
:1024000057FC074606E05CE0FFF752FCC11B494859
:10241000814256D8E8698007F6D40098002804D095
:10242000F16B012000078143F163E069002873D05C
:10243000B1688906490F02294DD001273F060228BD
:10244000306805D0B8433060FFF732FC04463AE00C
:10245000B8433060FFF72CFC054604E0FFF728FC8A
:10246000401B02282DD830688001F7D4616A206AA9
:10247000A26A0843E16A120211430843216B084330
:10248000F1682D4A11400843F060306838433060ED
:10249000F068012109070843F06000E03AE0FFF727
:1024A00007FC044604E0FFF703FC001B022808D8E1
:1024B00030688001F7D52FE0FFF7FAFB001B0228F8
:1024C00001D90320F8BD30688001F5D4F0681B49BC
:1024D0000840F06020E00128F4D0F068226A81070B
:1024E000890F914216D17021626A0140914211D147
:1024F0007F21A26A09020140120291420AD11F21E2
:102500004904E26A0140914204D1400F216B400727
:10251000884201D00120F8BD0020F8BD0010024023
:102520000024F4005C000020540000204010024011
:1025300000700040881300008C80C11FFCFFFEEF7C
:10254000094910B5401E884201D9012010BD074C31
:1025500060610321081F01F0B1FF0020A061072086
:102560002061002010BD0000FFFFFF0000E000E040
:1025700070B5040005D025462035687F002802D0BC
:1025800006E0012070BD00202877204600F016F8F4
:1025900002206877211D206801F008FA01224034EA
:1025A0002272AA77EA7722706270A270E2702271BA
:1025B0006271A271E2716A77002070BD08B500688F
:1025C0000549884207D105480268C9130A430260D9
:1025D00000680840009008BD002000404010024004
:1025E000014620314A7F012A01D001207047022292
:1025F0004A770168CB6801221343CB600068094920
:10260000884202D00849884207D18168074B1940A7
:10261000062905D0DB1F994202D0016811430160F1
:1026200000207047002C014000040040070001001A
:1026300010B586B0044614216846FDF79EFD0E498C
:102640002068884215D10D48416B01221143416336
:10265000406B6946104005901020009002200190C8
:102660000020029003900420049005200007FFF74B
:102670006BFA06B010BD00000020004000100240C0
:10268000F8B504460020264620360090307F0D46DF
:1026900001280CD00120082730770C2A48D008DC0C
:1026A000002A10D0042A1ED0082A06D130E00220C9
:1026B000F8BD102A52D0142A60D0012000900020CA
:1026C00030770098F8BD206801F0BCF92068816976
:1026D00039438161206881690422914381612068C6
:1026E00081692A6911E0206801F0EAF920688169AE
:1026F0000122D20211438161206881695210914305
:102700008161206881692A69120211438161D6E7DB
:10271000206801F015FA2068C1693943C161206859
:10272000C16904229143C1612068C1692A6912E02C
:10273000206801F045FA2068C1690122D2021143E4
:10274000C1612068C269012189028A43C26120688F
:10275000C1692A6912021143C161B0E7206801F022
:1027600065FA2068416D394341652068426D042156
:102770008A4342652068416D2A6912E0206801F0B1
:1027800083FA2068416D0122D2021143416520681D
:10279000426D012189028A4342652068416D2A69A0
:1027A0001202114341658AE770B5040005D0254641
:1027B0002035687F002802D006E0012070BD00208F
:1027C0002877204600F016F802206877211D20683F
:1027D00001F0ECF8012240342272AA77EA772270E5
:1027E0006270A270E27022716271A271E2716A7706
:1027F000002070BD7047000030B503460446002538
:102800002033403000290CD004290CD008290CD0EA
:102810000C290CD010290CD0C278012A0BD0012031
:1028200030BD9A7FF9E7DA7FF7E70278F5E742787B
:10283000F3E78278F1E70222002912D0042912D0AE
:10284000082912D00C2912D0102912D0C2700029E8
:1028500011D0042914D0082916D00C2940D0012504
:102860003CE09A77F3E7DA77F1E70270EFE742703E
:10287000EDE78270EBE72068C3681343C36008E0AC
:102880002068C268042302E02068C26808231A4353
:10289000C2600122206801F0C7F81349206888420D
:1028A00005D0124A904202D0114A904204D1426CA3
:1028B0000123DB031A43426420680122884202D0CC
:1028C0000C49884207D181680B4B1940062905D075
:1028D000DB1F994202D0016811430160284630BDD8
:1028E0002068C2681023D2E7002C01400044014058
:1028F00000480140000400400700010010B50146F7
:1029000080310A79012A15D001220A7124228A60B5
:102910000268136814686408640014600122520796
:1029200093430022426600680360202088600A7199
:10293000104610BD022010BD7047704770B50446A8
:1029400005468034207901281AD0012020712420E6
:10295000A060286806680268520852000260286871
:10296000826807235B069A430A438260284601F087
:10297000BDF9286806602020A0600020207170BD8D
:10298000022070BD70B504460546803420790128C8
:1029900019D0012020712420A060286806680268F0
:1029A00052085200026028688268D200D2080A43A6
:1029B0008260284601F09AF9286806602020A0600D
:1029C0000020207170BD022070BD70477047F8B5BF
:1029D00004468034A1680546E668006882681027CE
:1029E0001206002A1BDA212919D1EFF310810122E6
:1029F00082F31088826880239A43826081F3108872
:102A0000E86F002808D0FEF73DFD002804D0E86FED
:102A1000FEF7F2FD202824D0284601F00DFB28689F
:102A2000816849061BD5222E19D1EFF310810122AE
:102A300082F31088826840239A43826081F3108871
:102A40002068002808D0FEF71DFD002804D020686B
:102A5000FEF7D2FD202804D0284601F0BBFA002062
:102A6000F8BD27610320F8BD70B504001AD02420FA
:102A700025468035A8602068016849084900016042
:102A80002068002606602068466020688660204630
:102A900000F0BAF92E61AE60EE60E66626672E7130
:102AA000002070BD012070BD70470000F8B50368BC
:102AB0000446D86919689A68B44D06462E402546E2
:102AC0008035002E75D0B24EB24F16400F403743BE
:102AD0006ED0C70706D0CF0504D501271F622B692A
:102AE0003B432B61830708D5D30706D02768022311
:102AF0003B622B6904273B432B61430708D5D3076F
:102B000006D0276804233B622B6902273B432B61D5
:102B1000030709D520230B40334305D0266808233B
:102B200033622E691E432E61030509D54B0107D57B
:102B300001232668DB0233622B69202633432B6195
:102B40002B69002B42D080060AD520200140C00509
:102B50000240114304D0616F002901D0204688470C
:102B6000286921688968490602D42821084232D0A0
:102B7000204601F02FFA20688168490627D5EFF337
:102B80001081012282F3108883684022934383607E
:102B900081F310882868002819D07F49816328684C
:102BA000FEF7AAFC002811D02868816B0DE000E038
:102BB00017E0860615D5012720263F070E4017404F
:102BC0003E430ED0616FB5E020468847F8BD2046F1
:102BD000FFF76AFFF8BD2046FFF766FF0020286177
:102BE000F8BDE66E012E7DD1C6067BD5CE0679D521
:102BF00010221A622068816826464906403600295C
:102C000049DA2B68196849680904090CE8D0B78BC0
:102C10008F42E5D9F18319680968890634D4EFF346
:102C20001081012383F3108803681701BB430360FD
:102C300081F31088EFF31081012080F31088206861
:102C400083685B085B00836081F31088EFF3108179
:102C5000012080F31088206883684027BB4383608D
:102C600081F310882020E8600020E066EFF31081F7
:102C7000012080F31088206803689343036081F388
:102C800010882868FEF7FEFB02202067B08BF18BCE
:102C9000401A81B235E0B18BF38BC91AF38B89B23C
:102CA000002B9DD000299BD0EFF31083012686F3E3
:102CB00010880668FF272137BE43066083F310881B
:102CC000EFF31083012080F3108820688668304F6E
:102CD000FF433E40866083F310882020E860002098
:102CE000E06600E011E0EFF310836067012080F3FD
:102CF0001088206805689543056083F310880220DA
:102D000020672046FFF718FEF8BDC60208D5560218
:102D100006D50120000518622046FFF757FEF8BDD2
:102D200006060BD501278026FF050E403A401643C4
:102D300004D0A16F002900D046E7F8BD420614D5A3
:102D40004A0612D52046EFF31081012282F3108843
:102D50001A684024A2431A6081F310882021A960D8
:102D60000021816700F070F9F8BD020205D54A0024
:102D700003D52046FFF729FEF8BDC001FCD5002988
:102D8000FADA2046FFF7D9FDF8BD00000F08000071
:102D90000100001020010004613E000870B504002D
:102DA00005D025468035A868002802D006E001201D
:102DB00070BD00202871204600F048F82420A8604B
:102DC00020680168490849000160204601F052F975
:102DD0000128EDD0A06A002802D0204600F0A8FF0C
:102DE000206841680922D2029143416020688168CD
:102DF0002A22914381602068016801221143016009
:102E0000204600F0FBFF70BD10B5044600680C4979
:102E1000884213D10B48016801229203914301605B
:102E2000C0210948FEF778FD80200059FEF7A2FB7B
:102E3000E06FFEF79FFB1B20FEF79EFF10BD00001A
:102E4000003801404010024000040050F0B58DB041
:102E5000044614216846FDF790F9182105A8FDF7EE
:102E60008CF93249206888425ED101200026059005
:102E7000069605A8FEF7C6FF002801D0FDF776FFED
:102E80002B480268012189030A4302600068084058
:102E90000B9027484038426B02210A434263406B43
:102EA0006A4608400B90C02043C2039669462148F9
:102EB0000496FEF749FE214D1F482860AE6032207F
:102EC000EE60686080206E61AE6147012F62EE6146
:102ED00028612846FEF7F2FB002801D0FDF746FFE7
:102EE00080200551AC621448144D14305C352860C4
:102EF000332068601020EE60A8606E61AE612F62C2
:102F00008020EE6128612846FEF7D8FB002801D01A
:102F1000FDF72CFFE567002201211B20AC62FEF7C4
:102F200047FF1B20FEF738FF0DB0F0BD0038014011
:102F300040100240000400501C0002401C0600200B
:102F400070B58C231B58202B01D0022070BD0029A6
:102F50000BD0002A09D0012483682403A34206D1A0
:102F60000369002B03D1CB0701D0012070BD0023E2
:102F7000C36603685C6824020BD5EFF31084012557
:102F800085F310881D680126B60635431D6084F35D
:102F9000108801F025F970BD7047704770B505467F
:102FA00004468035A868202801D0022070BD002981
:102FB0000BD0002A09D00123A0681B03984206D138
:102FC0002069002803D1C80701D0012070BD204628
:102FD000403021658282C282002129612120A860BF
:102FE000E06F002819D0154BC362E36F14481863D3
:102FF000E36F14485863E06F134681632068E66FFF
:10300000024628323046216DFEF7AAFB002804D084
:10301000102028612020A860D7E72168402008629E
:10302000EFF31081012080F31088206882688023EC
:103030001A43826081F31088002070BD7D3F000834
:10304000C93F0008753E000870477047FEE770B53D
:1030500001240525E4022D07002221462846FEF71B
:1030600020FE6600002231462846FEF71AFE0220A6
:1030700001F0FCFA012221462846FEF712FE02204A
:1030800001F0F4FA002221462846FEF70AFE01224A
:1030900031462846FEF705FE70BD70B501240525B2
:1030A000E4022D07002221462846FEF7FAFD012200
:1030B000160331462846FEF7F4FD042001F0D6FA47
:1030C000012221462846FEF7ECFD042001F0CEFA4D
:1030D000002221462846FEF7E4FD0122314628461B
:1030E000FEF7DFFD70BDF1B500240126F6020527CD
:1030F00025463F07002231463846FEF7D2FD022022
:1031000001F0B4FA012231463846FEF7CAFD6006E6
:10311000040E012109033846FEF7B6FD002801D050
:10312000641CE4B2012001F0A1FA6D1CEDB2082D7F
:10313000E0D30098002803D0FFF789FF2046F8BDB0
:10314000FFF7ABFFFAE7F8B5012605270546F602BB
:103150003F07002231463846FEF7A3FD0024E80968
:1031600001D0012200E00022012109033846FEF7C8
:1031700098FD6806050E022001F078FA012231461A
:103180003846FEF78EFD022001F070FA002231462B
:103190003846FEF786FD022001F068FA641CE4B2AE
:1031A000082CDCD3F8BD70B50122052514032D07CA
:1031B00021462846FEF775FD0122D60231462846F3
:1031C000FEF76FFD042001F051FA00222146284647
:1031D000FEF767FD042001F049FA00223146284637
:1031E000FEF75FFD70BD70B501240525E4022D07D3
:1031F000002221462846FEF754FD66000022314693
:103200002846FEF74EFD042001F030FA0122214647
:103210002846FEF746FD012231462846FEF741FDCD
:10322000042001F023FA70BDF8B50122052516032C
:103230002D07002431462846FEF733FD012001F01A
:1032400015FA0122D70239462846FEF72AFD012049
:1032500001F00CFA07E0641CE4B2642C03D9FFF718
:10326000C2FF0120F8BD31462846FEF70DFD0028BB
:10327000F1D1002239462846FEF713FD0020F8BDA3
:103280008068C007C00F704780684007C00F704754
:10329000C0680005800F01D00020704701207047F2
:1032A000026807239B059A430A430260704710B5E2
:1032B00043690424214007248C40A3438A401343DC
:1032C000436110BDF8B55148418880884EBA45BA6F
:1032D00006214E4801F098F9010AC7B24C48009106
:1032E000028A4C494A80022282568A800279CA8028
:1032F000028B0A81428B4A81828B8A81C28BCA816E
:10330000428C0A828279437912021A434A82C28A23
:103310008A82808CC88270190C2833D83B48817906
:10332000B9422FD1C27900998A422BD10146027845
:1033300080390A7040784870680088700324002043
:103340000EE031184A003349895A304A0B12803A4C
:103350001355641CE3B2D1545B1C401CDCB2C0B2F8
:10336000A842EED329482146803801F04DF9274A7A
:10337000803A1055641CE1B2000A5054491CC8B28E
:1033800001F0AAF9FF2E1DD1012D3DD11F488179F1
:10339000B94239D1C1790098814235D1002405E084
:1033A000015D1A4880380155641CE4B21848303079
:1033B000FCF7EEFEA0421848F2D8FCF7E9FEC0B2D6
:1033C00001F08AF9FE2E1FD110488179B9421BD134
:1033D000C27900998A4217D104460178803C217055
:1033E000407860706800A0700948018C090AE1709B
:1033F000008C20710521204601F006F96071000A59
:10340000A071072001F068F9F8BD000060010020FC
:1034100000000020D403002030000020F8B57B4ECF
:103420000621B08840BA04B2708845BA304601F02F
:10343000EBF8034600203246803A315C1154401CC0
:10344000C0B20628F9D3D9B2180A9171704FD07161
:103450000F2D21D0042D46D06E4A5300052D5DD08E
:10346000062D7DD0072D7CD0082D7BD06A4A0A2DF1
:1034700079D00B2D0FD1B37999420CD1F1798842D3
:1034800009D1944207D824257D5FBC8401F0E0FA7D
:10349000002824D0BD84F8BDB3799942FBD1F179DD
:1034A0008842F8D1601EF6280CD8F889FC81C5B294
:1034B00001F0CEFA002801D0FD81F8BD7078002817
:1034C0000DD1F8BDFF2010715071144606214F48F0
:1034D00001F09AF8A071000AE0713078EFE7082057
:1034E00001F0FAF8F8BDB2799142FBD1F179884246
:1034F000F8D17D20C0008442F4D8388B3C8305B2DB
:1035000001F0A6FA002801D03D83F8BD082001F0A3
:10351000E3F8388B414909684863F8BDB579A94299
:10352000FBD1F1798842F8D1A0189842F5D81A2534
:103530007D5F20460A2148431021795EFCF7F0FDAB
:103540007883601F0F2800D87C831A20385E0528F6
:10355000E3DB1A20385E1428DFDC01F079FA03E09F
:1035600006E017E028E040E00028B8D07D83F8BDF1
:10357000B579A942FBD1F1798842F8D1A0189842D7
:10358000F5D81C257D5FBC8301F062FA0028A6D027
:10359000BD83F8BDB2799142FBD1F1798842F8D16F
:1035A000FD8BFC831E48B8620020388401F05AFA73
:1035B000002894D0FD83F8BDB2799142FBD1F17916
:1035C0008842F8D1032CF6D822257D5F7C8401F057
:1035D0003FFA002801D07D84F8BD082001F07CF876
:1035E0002220385E00F0ECFEF8BDB3799942FBD1A1
:1035F000F1798842F8D19442F6D816257D5FFC8295
:1036000001F026FA0028B0D0FD82F8BD600100204C
:1036100000000020E40C0000DC0500003C05002058
:10362000D87700083EB50021184800910191164A4C
:10363000029102600122D20481604260C1601203E3
:10364000026104224261017641760124847641625E
:103650000246C46120328162117307234363016310
:103660001177C164FDF70CFD002801D0FDF77EFB4A
:1036700007480090694601940448FDF7EDFB0028D7
:1036800001D0FDF773FB3EBD002401406C04002017
:103690000200000408B50C48816B012211438163CC
:1036A000806B02211040009000220920FEF780FB71
:1036B0000920FEF771FB002202210A20FEF778FBA9
:1036C0000A20FEF769FB08BD00100240F0B587B084
:1036D00014216846FCF751FD3C48416B02263143FA
:1036E0004163416B31400591416B012529434163A1
:1036F000406B2A4628400590052035490007FEF713
:10370000D0FA0520002220210007FEF7CAFA314F27
:10371000012211463846FEF7C4FA04200024009026
:10372000052002946946019503940007FEF70CFA00
:103730000820009031200004019005206946029481
:103740000007FEF701FA2020009005206946039645
:10375000019502940007FEF7F7F94020009005203C
:103760000194694602940007FEF7EEF9802000906C
:103770001120000401900520694602940007FEF71D
:10378000E3F9009502946946384601950394FEF7E3
:10379000DBF90320C0020090112001AA51C20520CC
:1037A00069460007FEF7D0F9002202210620FEF745
:1037B000FFFA0620FEF7F0FA002202210720FEF7AA
:1037C000F7FA0720FEF7E8FA07B0F0BD0010024054
:1037D000041800000004005010B588B01C21684691
:1037E000FCF7CBFC174816490160002402218460D5
:1037F0004160046114498461C160FEF7B9FE00288C
:1038000001D0FDF7B3FA0F48FEF7CEFF002801D034
:10381000FDF7ACFA602000907D20C000019002947A
:103820000022694604940748FEF72AFF002801D0C9
:10383000FDF79CFA0348FEF7FBFE08B010BD000040
:10384000002000403C050020E703000010B51848A8
:10385000164901604B21C901416000218160C160AE
:1038600001618161C16101620C2241624261816238
:10387000FFF794FA002801D0FDF778FA00210C48F0
:10388000FFF780F8002801D0FDF770FA0021084802
:10389000FFF754F8002801D0FDF768FA0448FFF755
:1038A0002DF8002801D0FDF761FA10BD0038014065
:1038B00088050020FEE77047704710B5FEF706FA4E
:1038C00000F002F810BD000030B5184B5868012414
:1038D000002804D05868401E586000D11C70144D58
:1038E00000210C20484340194268002A09D0426850
:1038F000521E426005D144700278012A01D18268CB
:103900004260491CC9B20629EBD39868401C9860F4
:103910009868084A0021904200D199605878401C6C
:10392000C0B258700A2800D3597030BD440000203E
:10393000EC030020FFFFFF7F30B591B034216846D3
:10394000FCF71BFC002401200D940E940F94400200
:103950001094FEF731FA0A200090FF200130039006
:10396000402005900120069008200A90022580033F
:103970000B900795000304940C90089509946846F1
:10398000FEF7F6FB002801D072B6FEE707200D9087
:103990000F9402210E9510940DA8FEF7E3FA00286B
:1039A00001D072B6FEE711B030BD704770B5026845
:1039B000184C194EA04201D0B04204D113467025D4
:1039C0004A68AB431A43154B154DA04208D0B0428C
:1039D00006D0144EB04203D0984201D0A84204D180
:1039E00003263602B243CE6832438026B2434E6984
:1039F000324302608A68C2620A688262A04203D0CF
:103A0000984201D0A84201D10969016301214161B5
:103A100070BD0000002C0140000400400044014043
:103A2000004801400020004010B5C906C90E01231E
:103A3000046A8B409C430462036A8A401343036216
:103A400010BD0000F0B5026A520852000262056A19
:103A500043688269164C174E224092080C68920007
:103A60001443022295438A68134F2A43B04204D07C
:103A7000B84202D0114DA84206D10825AA43CD680C
:103A80001543042295432A46B04204D0B84202D0DE
:103A90000A4DA84206D103252D02AB434D691D43B3
:103AA0008B692B4343608461496841630262F0BDC6
:103AB0008FFFFEFF002C0140004401400048014000
:103AC000F0B5026A10239A430262046A436882696D
:103AD000174D184E2A4003252D02AA430D682D02CA
:103AE0001543202294438A6812012243B04207D131
:103AF0001446CA688027BC43120122434024A243D3
:103B0000B04205D00C4CA04202D00C4CA04208D1CF
:103B10000324A402A3434C69A4001C438B699B00AB
:103B2000234343608561496881630262F0BD000000
:103B3000FF8FFFFE002C014000440140004801407F
:103B4000F0B5026AFF2301339A430262046A4368B4
:103B5000C269174D174E2A4092080D68920015430E
:103B60000122520294438A6812022243B04207D1D2
:103B70001446CA68C714BC43120222430415A24368
:103B8000B04205D00C4CA04202D00C4CA04208D14F
:103B900003242403A3434C6924011C438B691B01A8
:103BA00023434360C5614968C1630262F0BD000000
:103BB0008FFFFEFF002C01400044014000480140FF
:103BC00070B5026A01231B039A430262046A4268C9
:103BD000C369124D2B4003252D02AB430D682D0206
:103BE0001D4301235B039C438B681E030C4B264340
:103BF000984205D00B4B984202D00B4B984206D10D
:103C000001241346A4034A69A34392011A43426064
:103C1000C56149680164066270BD0000FF8FFFFE48
:103C2000002C0140004401400048014070B5026A88
:103C300001263604B2430262036A4268446D0E4DA7
:103C40002C400D6825437400A3430C8924041C43B5
:103C50000A4B984205D00A4B984202D0094B984231
:103C600004D113464A69B34312021A4342604565C0
:103C700049688165046270BD8FFFFEFF002C014022
:103C8000004401400048014070B5026A01231B0551
:103C90009A430262036A4268446D104D2C400D68DD
:103CA0002D02254301246405A3430C8924051C43EC
:103CB0000B4B984205D00B4B984202D00A4B9842CE
:103CC00006D101261346B6044A69B34392021A4349
:103CD000426045654968C165046270BDFF8FFFFEA3
:103CE000002C01400044014000480140F8B5044662
:103CF000416E4034002915D0006881688068090150
:103D00004D0F0A4E400F3746315C083F385CC0000B
:103D1000FCF7F0F96085785D715DC000FCF7EAF9A9
:103D20002085F8BD01206085FAE70000B04B00084F
:103D300010B5018DC90707D001684A6801235B04EB
:103D40009A43C36A1A434A60018D890707D50168FF
:103D50004A6801231B049A43036B1A434A60018D8E
:103D6000490707D501684A6801239B049A43436BBE
:103D70001A434A60018D090707D501684A68012383
:103D8000DB039A43836B1A434A60018DC90607D54A
:103D900001688A6801231B039A43C36B1A438A6034
:103DA000018D890607D501688A6801235B039A4360
:103DB000036C1A438A60018D490612D501684B686D
:103DC00001221205446C934323434B60416C9142A2
:103DD00007D101684A6803235B059A43836C1A4341
:103DE0004A60018D090607D501684A680123DB0492
:103DF000C06C9A4302434A6010BD0000FEB5054600
:103E00000026803504462E61FDF752FF01902068A0
:103E10000068124F000709D50121009700224905CB
:103E20002046019B00F034FA00280DD1206800687C
:103E300040070BD501210097002289052046019BF0
:103E400000F026FA002801D00320FEBD2020A86043
:103E5000E860E66626672E710020FEBDFFFFFF01C9
:103E600010B5806A002201464031CA83CA82FEF73B
:103E70001BFE10BDF8B5846A204680308168054677
:103E8000C6682068806800270006002806DA212915
:103E900004D156200753204600F0CEF820688068F1
:103EA000400606D5222E04D15E200753204600F09E
:103EB00091F828691021084328612046FEF7F4FD97
:103EC000F8BD70B501460968806A09680023890653
:103ED000002937DB5E210B52EFF31082012181F3C1
:103EE000108801680C68FF250135AC430C6082F333
:103EF0001088EFF31082012181F3108801688C682B
:103F0000640864008C6082F31088EFF31082012152
:103F100081F3108801688C684025AC438C6082F383
:103F2000108820228C210A50C16E01290AD1EFF39A
:103F3000108281F3108801680C681025AC430C6076
:103F400082F310880367C16E012902D0FFF724F8BD
:103F500070BD5C21095AFEF7EFFC70BD10B5806A98
:103F600001210167C16E012902D0FFF716F810BDCB
:103F70005C21095A4908FEF7DFFC10BD10B5014667
:103F80000968806A096889061BD4002256210A52F2
:103F9000EFF31082012181F3108801688B6880247F
:103FA000A3438B6082F31088EFF31081012282F328
:103FB00010880068026840231A43026081F3108869
:103FC00010BDFFF741F810BD10B5806AFFF73DF84E
:103FD00010BD000010B5EFF31082012181F31088AD
:103FE00001680B68FF242134A3430B6082F310881F
:103FF000EFF31082012181F3108801688B680D4C6A
:1040000023408B6082F31088C16E01290AD1EFF33F
:10401000108281F3108801680B681024A3430B60A1
:1040200082F3108820228C210A500021C16641674A
:1040300010BD0000FEFFFFEF10B5EFF3108201216D
:1040400081F3108801680B68C024A3430B6082F3DE
:104050001088EFF31082012181F3108801688B68CA
:104060000124E405A3438B6082F310882021803073
:10407000816010BDF8B5044681680069E2690143BA
:104080006069002510430143206802684C4B1A40C8
:104090000A43026020684168032212039143E268E8
:1040A00011434160216AA069014320688268454B41
:1040B0001A400A4382602068C16A626A09090901DC
:1040C0001143C1624049206888420FD13F4840698E
:1040D0008007800F10D0012804D002280CD00328BC
:1040E00009D101E0042007E0082005E038498842B2
:1040F00001D1002000E010200122E369D2033549FC
:10410000354E364F93422AD1002806D0022807D0D8
:10411000042807D0082843D108E0FDF7CFFF03E0CB
:104120000A4603E0FDF7DEFF02003ED0606A400071
:10413000315A1046FBF7DEFF616840004A088018DC
:10414000FBF7D8FF01461039B94229D82349491C49
:1041500001400007420F20680A43C26025E00028A2
:1041600006D0022807D0042807D0082818D108E074
:10417000FDF7A4FF03E00A4603E0FDF7B3FF0200EA
:1041800013D0606A4000315A1046FBF7B3FF6168F4
:104190004A088018FBF7AEFF01461039B94201D931
:1041A000012502E0216880B2C8602046012140302C
:1041B0004185018500206067A0672846F8BD0000A2
:1041C000F369FFCFFFF4FF110038014040100240B7
:1041D000004400400024F400904B0008EFFF000072
:1041E00070B50446816540300021254682838035C4
:1041F00029612220E8602868002819D0214BC36279
:104200002B68214818632B68204858632868134698
:104210008163A66D2168324624312868FDF7A0FA33
:10422000002805D0102028612020E860012070BD02
:10423000206900280CD0EFF31081012080F3108852
:1042400020680268FF2301331A43026081F310885B
:10425000EFF31081012080F3108820688368012229
:104260001343836081F31088EFF3108182F3108889
:104270002068826840231A43826081F310880020FE
:1042800070BD0000C33E00085D3F0008753E000899
:10429000FFB581B005460F46044680350A9E54E0BE
:1042A000701C52D0FDF704FD0499401AB0422FD87B
:1042B000002E2DD020680168490746D5C069C0434B
:1042C000000542D401202168C0020862EFF310818A
:1042D000012080F3108820680268FF23A1339A43ED
:1042E000026081F31088EFF31081012080F31088C1
:1042F0002068826852085200826081F31088202072
:10430000A860E860286100202871032005B0F0BD96
:10431000EFF31081012080F3108820680268FF23EA
:10432000A1339A43026081F31088EFF310810120DA
:1043300080F310882068826852085200826081F3FE
:1043400010882020A860E860DDE72068C169384651
:10435000884305D0002003998842A1D00020D5E7EA
:104360000120F8E710B51148FEF7A0FB0F48FEF753
:104370002EFB0E480068C169C943C90610D410213C
:1043800001620B48017800290AD10A490968496885
:104390008022511A0170027807490848FBF7D4FEC1
:1043A000802205490148FEF7CBFD10BD880500209D
:1043B000000000201C06002060000020600100209A
:1043C00010B504461F48FEF74FFB1E491E48086003
:1043D0004B20C0014860012C02D0022C03D005E024
:1043E0004B20000201E0E1200002486000208860CC
:1043F000C86008618861C86108620C2248624A612D
:1044000088621048FEF7CAFC002801D0FCF7AEFC19
:1044100000210C48FEF7B6FA002801D0FCF7A6FCF4
:1044200000210848FEF78AFA002801D0FCF79EFC1C
:104430000448FEF763FA002801D0FCF797FC00F06F
:104440006DF910BD880500200038014010B50D48F9
:104450000D4A0178D3894078994202D11378082B0C
:1044600005D0002902D11178082902D010BD0328F7
:1044700004D00628FAD1FEF7D1FF10BDFEF722FFC7
:1044800010BD000060010020000000202021020C6F
:1044900001D010211046020A01D010460839020945
:1044A00001D01046091F820801D01046891E42081B
:1044B00001D0881E7047081A704700008307FF224A
:1044C000DB0E9A408907090E9940002808DB830813
:1044D00009489B001818036893430B430360704717
:1044E0000007000F0838830804489B001818C369A8
:1044F00093430B43C361704700E400E000ED00E02C
:1045000002E008C8121F08C1002AFAD1704770479C
:10451000002001E001C1121F002AFBD170470000FA
:10452000062806D20C214843054940184178012944
:1045300001D0002070470021417001207047000029
:10454000EC03002070B50020154B04460C214143BC
:104550000A46C9184C608C604C709C54401CC0B218
:104560000628F3D30F487D21C9000068FBF7C2FD80
:104570000D49401E884201D901200CE00B494861D9
:104580000B480722C3691B021B0A4D042B43C3615E
:104590008C610A610020002800D0FEE770BD000099
:1045A000EC0300205C000020FFFFFF0000E000E0C3
:1045B00004ED00E0062800D3FEE7012282F3108814
:1045C0000C22064B5043C21851609160002151707B
:1045D00001221A5481F3108870470000EC03002078
:1045E000062800D3FEE7012181F310880C21054B3A
:1045F00000224843C1184A604A701A5482F3108856
:1046000070470000EC03002030B503460B480C4C0B
:104610000DE01A78504000225B1CC50702D040080C
:10462000604000E04008521CD2B2082AF5D30A4686
:10463000491E89B2002AECD130BD0000FFFF000006
:1046400001A0000000280ED0012800D10220012185
:1046500081F31088044948600020087080F31088B6
:1046600008780128FCD1704744000020F8B50D4EB1
:104670000746756900240D480B490068FBF73AFDB1
:104680007843B1690246B0698842FCD0884201D2C1
:10469000091A01E02B1A59180C1901469442F2D359
:1046A000F8BD000000E000E040420F005C00002088
:1046B000FDF714FBFFF740F9FFF744FFFFF706F89B
:1046C000FEF7E8FFFEF7AEFFFFF786F8FFF7BEF84C
:1046D00000F03CF8FEE7000070B5052504462D0704
:1046E000012220212846FDF7DCFA22460849094824
:1046F000FEF754FC0848FCF781FF0128FAD1052099
:10470000FFF7A0FF002220212846FDF7CAFA70BD5E
:10471000E0000020880500207806002010B5094937
:104720000868026810231A43026009685020086272
:10473000FFF708FF7D21382209010348FCF716FA2C
:1047400010BD00008805002034040020FFF7E6FFBC
:10475000A04EA148318801800188A04C002902D0D8
:104760000188A14201D1012101809D487188018009
:104770000188002902D00188A14202D1AF2189001D
:10478000018000889749096848639748B18801808B
:104790000188002903D00021415E491C01D10A2172
:1047A00001809248F188018001880025002902D00B
:1047B000415F491C00D105808D49308908800888F7
:1047C000002803D00020085E401C00D10D8000208E
:1047D000085EFFF7F5FD874871890180018800298F
:1047E00003D00021415E491C01D1282101800C2009
:1047F000305E81490028088001D0401C02D1FF2092
:104800002D3008807D487E4B724F7E4C303F0146F4
:1048100018600888208008892288002A03D026880A
:104820006E4A964200D12580002802D06B4A904201
:1048300000D100202288904205D9B94203D82080B7
:1048400008311960E5E76748FDF7CAFE00216548B1
:10485000FDF7D2FF6C48FEF7BAF880226B496A4830
:10486000FEF76EFBFA226A496A48FCF775FD0520DF
:10487000002220210007FDF714FA32210020FFF763
:1048800099FEFF21F5310120FFF794FE62490320D4
:10489000FFF790FE7D21C9000420FFF78BFE0A215F
:1048A0000520FFF787FE00260020FFF739FE0028CD
:1048B00009D05848FCF7AAFDFCF780F8FA225449C1
:1048C0005448FCF749FD0120FFF72AFE002808D0D4
:1048D000524805805248FDF7F1F901215148FDF792
:1048E000D8F90220FFF71CFE00283AD0761C0520DC
:1048F000B6B204210007FDF7CCF9E1204001864261
:104900002FD92088401C208021883448814200D142
:104910002580454800781E2806D8FBF71BFE434A31
:10492000434BFBF793FD0AE04042FBF7FFFD3F4A94
:104930003F4BFBF78BFD00223E4BFBF7D3FC0646BB
:104940003D480F460078FBF705FE32463B46FBF735
:1049500023FE03D839480188491C018000F082F801
:1049600000260320FFF7DCFD002802D03449022096
:1049700008700420FFF7D4FD00280BD00220FFF7B9
:104980002FFE0520012204210007FDF78AF92D4999
:10499000012008700520FFF7C3FD002810D02A4829
:1049A000FCF772F8284F7879022809D1386BFBF7A9
:1049B000DFFD21490870786BFBF7DAFD1A490870B2
:1049C000224F3878002800D16EE7FFF73FFD3D7099
:1049D0006AE70000007800080E000020FFFF0000DA
:1049E000180000203C0500201A0000201C000020B8
:1049F0002200002016000020240000200070000883
:104A0000280000201E0000208805002060000020F3
:104A1000E00100206C040020881300004200002008
:104A20002C0500200004005005000020CDCCCCCC8B
:104A3000CCCC06400080664006000020200000200C
:104A400002000020040000203404002000000020A8
:104A500010B5012080F3108800F03CF8002181F3AC
:104A6000108810BD10B586B002200090042001907F
:104A70000E2002900120144C0390A06A0830A0621E
:104A8000FCF736FF1149A06A88420CD91048A06291
:104A900004A96846FCF7AAFE002804D0FCF7EAFE49
:104AA000012006B010BDE28B00230120A16AFCF7B3
:104AB000EFFE002803D0FCF7DDFE0320F1E7FCF752
:104AC000D9FE0020EDE7000000000020D8770008A4
:104AD0000070000800B589B000200090019002909D
:104AE000039002200490042005900F2006900120DE
:104AF00007902548C1896A461170C189090A517019
:104B0000018B9170018B090AD170418B1171418B1E
:104B100009125171818B9171818B0912D171418C74
:104B20001172418C09125172C18A9172C18A0912A3
:104B3000D172808C107300125073FCF7D9FE08A953
:104B400004A8FCF753FE002804D0FCF793FE0120D4
:104B500009B000BD0D490120019B009AFCF798FEA9
:104B6000002808D1094901200831039B029AFCF76B
:104B70008FFE002803D0FCF77DFE0320E8E7FCF75A
:104B800079FE0020E4E70000000000200078000823
:104B9000010002000400060008000A000C001000DA
:104BA0002000400080000001010101030701000016
:104BB00008040204080101010000000000000000D8
:104BC00000000000000000000000000000000000E5
:104BD00000000000000000000100000002000000D2
:104BE00003000000040000000600000007000000B1
:104BF00008000000090000000000000000000000A4
:104C000000000000000000000100000002000000A1
:104C10000300000004000000384C000800000020E1
:104C20006000000000450008984C0008600000206B
:104C3000900A00001045000800010100010000007A
:104C4000000000000000000000000000000028003C
:104C50000000000000000000000000002C01000027
:104C600000700008000000004443452D323430330A
:104C70002D56352E325F48414C00000000000000E8
:104C8000000000000000000001000000040000001F
:084C9000000000000024F40004
:04000005080000C12E
:00000001FF
